:020000040000FA
:020000000C28CA
:08000800A00105080939083CBC
:100010000319A00A0B100900831600308100093073
:10002000850050309F00073095001614831207306A
:10003000990000309F000630850083160515831255
:10004000051D852A8316051183120030EE22A400B7
:100050000030A00006308500C8308B0083160515DF
:100060008312051DBA2A201C31288B018316051125
:100070008312A001851085193B288316051483126D
:100080000511851D4128851480300518A00405152B
:10009000851948280511851D4B2885104030051805
:1000A000A0040515851952280511851D55288514AC
:1000B00020300518A004051585195C280511851D3B
:1000C0005F28851010300518A004051585196628CD
:1000D0000511851D6928851008300518A00405152F
:1000E000851970280511851D7328851004300518A1
:1000F000A004051585197A280511851D7D28851010
:1001000002300518A0040515851984280511851DE0
:1001100087280130051C8E28A00485142008A10022
:10012000F030A005A03020060319B228C030A00589
:100130000319A728851005118422051584220511AD
:100140008422051584220511842285142C28051586
:100150008519A828051083160510831205100511AE
:100160003F30BB2805158519B328051083160510E7
:10017000831205110F30A105851DBC280515210826
:10018000A300A418A31724182317A30CA31324193E
:10019000A317031C352905118316851483128519AD
:1001A000CF280510851805140515851DD52883222F
:1001B00005118519D9280510851805140515851D03
:1001C000DF28832205118519E328051085180514F9
:1001D0000515851DE928832205118519ED280510CF
:1001E000851805140515851DF32883220511851929
:1001F000F7280510851805140515851DFD2883228F
:100200000511851901290510851805140515851D89
:1002100007298322051185190B2905108518051456
:100220000515851D1129832205118519152905102C
:10023000851805140515851D1B29832205118519AF
:100240001F298316051483120515842205118422A3
:10025000851083168510831285108422051584224B
:1002600085148316051483122C28851935298316C5
:1002700005148312A001051183228514A31F851084
:1002800083220515851D4229051180300518A0041B
:100290008514231F85108322051585194D29051105
:1002A00083228514A31E851083220515851D5629DA
:1002B0008322051140300518A0048514231E8510E3
:1002C0008322051585196229051183228514A31D32
:1002D000851083220515851D6B2983220511203089
:1002E0000518A0048514231D851083220515851982
:1002F0007729051183228514A31C851083220515F7
:10030000851D80298322051110300518A00485144D
:10031000231C85108322051585198C29051184223B
:10032000851084220515851D9329051108300518AF
:10033000A0048514A01F8510051585199D29051198
:1003400083228514201F851083220515851DA6296B
:100350008322051104300518A0048514A01E851001
:10036000832205158519B229051183228514201EC3
:10037000851083220515851DBB29832205110230B6
:100380000518A0048514A01D851083220515851964
:10039000C729051183228514201D85108322051588
:1003A000851DD0298322051101300518A00485146C
:1003B000A01C8510832205158519DC2905108316DC
:1003C00005108312051183228514201C85108322B9
:1003D0000515851DE92984220511842283168514BB
:1003E0008312832205158519F329051184228316AA
:1003F00005148312851DFA2905080939A00005088E
:100400000939A10020020319FF29A11D112A051590
:10041000842285108316851083128510211C3628AE
:100420002C288514831685108312201C85108422A5
:10043000051584220511851D1B2A8514051C8510B0
:10044000842205158519222A05118422851D262A54
:100450008514051C85108422051585192D2A051182
:100460008422851D312A8514051C851084220515DA
:100470008519382A05118422851D3C2A8514051CFE
:100480008510842205158519432A05118422851DAE
:10049000472A8514051C85108422051585194E2AC6
:1004A00005118422851D522A8514051C851084227D
:1004B00005158519592A05118422851D5D2A851483
:1004C000051C8510842205158519642A05118422CE
:1004D0000510831605108312831685148312851D5B
:1004E0006F2A8519712A8316051483120515842233
:1004F0000511832285108316851083128422051529
:10050000842285142C280800832A83160510831260
:100510000514E222051D892AE222831605118312A1
:100520000030EE22013E0739A400023EA500003053
:10053000F322831605118312A50B9F2AA72A0515FE
:10054000E822051D892A0511E82205159C2A2408A0
:10055000023EA500E822051D892AE822051D892AF8
:10056000E822051D892AE822051D892AE8220519A5
:100570009C2A892AE222051DBA2AE2228316051145
:100580008312E822E8220030EE220739013EA4005F
:10059000013EA500E822E822A50BCF2A2228051556
:1005A000E8220511E8220515CC2A1430A600000027
:1005B0000000A60BD72A08000A30A700D522A70BF7
:1005C000DE2A08001430A800DC22A80BE42A080068
:1005D0003230A900E222A90BEA2A080083169B0008
:1005E0001C141A08022B83169B00831224088316FE
:1005F0009A001C1555309D00AA309D009C149C1833
:10060000FF2A1C1183120000080053002E00200056
:100610004C00690063006800740065006E006200B1
:100620006500720067006500720020002D00200048
:10063000560065007200730069006F006E002000B4
:1006400033002E00310020006400750020003900C6
:100650002F00300035002F0030003600200046000B
:1006600058003100340020002D00200046005800C2
:1006700031003800200068007400740070003A00F7
:100680002F002F006C006900630068007400650093
:100690006E006200650072006700650072002E0047
:1006A00073002E0066007200650065002E00660073
:0206B0007200D6
:02400E00D23F9F
:024200000000BC
:00000001FF
